:020000040000FA
:10000000000083018A017928F1000308F2008312BD
:10001000031383130B1915208C1A37200C1A652033
:1000200072088300F10E710E09000B1106182328C7
:10003000B80A03192128B80A03192128B80A031D90
:100040002628B80326283808031DB8038619332844
:10005000B90A03193128B90A03193128B90A031D4D
:100060003628B90336283908031DB9030800981C3F
:100070003B281812181618196328361849281A0828
:10008000023C031D642836140511B3011330B5007A
:1000900064280408F3003308203E84001A08800016
:1000A000B200B30A3308023A031D5B2821080F3956
:1000B000B5000430B50735083306031D6428B614AF
:1000C0003610051564281A080800600803197028FE
:1000D0006208840000089900E003E20AE21278282E
:1000E0008316031383130C128312031383138514D3
:1000F000080015214E218B176400BC2081208D2023
:100100007C28F70185197714051AF7143A08770641
:10011000031908007708BA009928F701B81B77146B
:10012000B91BF7143B087706031908007708BB00D2
:1001300099280230A521E6010330F700770EE60783
:10014000A521630E033EE607A521A1210330E607A2
:10015000A521F701051B7714851BF71405187715E2
:100160007708E607A5213B08E607A5213A08E60738
:10017000A521E609660AA529B61C0800B6103208B2
:10018000B4003308F700F703203084000008B407F8
:10019000840AF70BC6283408031DDC2820080F3911
:1001A000033A031D5A292208013A0319DD282208BF
:1001B000023A0319EF28BA290800B201200EA00064
:1001C000B2070F30A105630E2104A100B207A121DF
:1001D0002208B2072308B207B209B20A5A29B201AB
:1001E000200EA000B2070630A100630E2104B20762
:1001F000A100A1210230B207A2005230B207A30031
:100200004530B207A4004C30B207A5002030B20739
:10021000A6005630B207A7003130B207A800B209D5
:10022000B20A0A30B500B3005A298313850186014A
:1002300083160313831368308F0083120317831709
:1002400016308500831603138313043081000730B2
:100250009C0000309B0038308500DF30860018128B
:100260001815333099008C169816831203138313D4
:100270000B178B169817181685140515B601B301C0
:10028000E001E3014030E100E200FF30BB00BA00D2
:100290001B30F8007121B700D32108000A30F700A5
:1002A0006400C83068218510C83068218514F70BB8
:1002B000502908000230A521B401B30320303407CF
:1002C00084000008A521B40AB30B5E293208A529D1
:1002D000F500FA30F6000000F60B6B29F50B6929E2
:1002E000080078088312031783178D0083160317FD
:1002F00083178C130C148312031783170C088312B3
:10030000031383130800F9008316031783178C184F
:10031000872983120317831778088D0079088C00CA
:100320008316031783178C130C158B1355308D0010
:10033000AA308D008C148B170C11831203138313B6
:100340000800E30A631AE30E0800E4006008203A9C
:100350000319A6296108840064088000E10AE112FB
:10036000E00A8316031383130C16831203138313FB
:10037000851008002208033A0319C2292208043A0A
:100380000319E1291B30F8000730A3050730A40545
:1003900023090739B70524082305B7043708832143
:1003A0003708D321E129F700771C051377180517C3
:1003B000F71C8513F7188517771D05107719051495
:1003C0000800B201200EA000B2070330A100630EA6
:1003D0002104B207A100A1212208B207F701051BE1
:1003E0007714851BF714051877157708A300B20753
:1003F000F701B81B7714B91BF7147708A400B207EC
:10040000F70185197714051AF7147708A500B207C4
:0C041000B209B20A0730B500B3005A2947
:02400E003C3F35
:02401000FC3F73
:00000001FF
